:1000000000308A0049290000FF00030E8301A1008F
:100010007F08A0000A08A8008A01A00E0408A20018
:100020007708A3007808A4007908A5007A08A6003C
:100030007B08A700831383128B1E20280B193328FB
:10004000220884002308F7002408F8002508F90096
:100050002608FA002708FB0028088A00210E8300E2
:10006000FF0E7F0E09008A1171283108F801300255
:1000700003183D283008F7004928F7010830B2007E
:10008000B00DF70D310877020318F700F80DB20B29
:1000900040288A117E28F701F80130080310311832
:1000A000F707F70CF80CB118F707F70CF80C311933
:1000B000F707F70CF80CB119F707F70CF80C311A21
:1000C000F707F70CF80CB11AF707F70CF80C311B0F
:1000D000F707F70CF80CB11BF707F70CF80C8A11AF
:1000E00085282908093C031C79282908AE00AF019E
:1000F00088282908B0000A30B10035287808AF00F8
:100100002F08B0000A30B1004B2878082902AE0051
:100110008316851083128510831605118312051529
:100120002E0B972883168601F330831286002E0843
:10013000023C031DA02883168601493083128600E5
:100140002E08033C031DA928831686016130831203
:1001500086002E08043C031DB22883168601333026
:10016000831286002E08053C031DBB2883168601DA
:100170002530831286002E08063C031DC4288316F2
:1001800086010530831286002E08073C031DCD280A
:1001900083168601F130831286002E08083C031D69
:1001A000D628831686010130831286002E08093C6A
:1001B000031DDF2883168601213083128600AE08D6
:1001C000031DE7288316860181308312860083167B
:1001D00005118312051183168510831285142F0BC8
:1001E000F62883168601F330831286002F08023C1E
:1001F000031DFF28831686014930831286002F08CD
:10020000033C031D08298316860161308312860092
:100210002F08043C031D11298316860133308312F5
:1002200086002F08053C031D1A29831686012530F8
:10023000831286002F08063C031D2329831686019E
:100240000530831286002F08073C031D2C298316D6
:100250008601F130831286002F08083C031D3529E2
:10026000831686010130831286002F08093C031D86
:100270003E2983168601213083128600AF08031DB4
:100280004629831686018130831286000B118A115C
:10029000202884011F308305703083168F001F12C1
:1002A0009F121B0880399B0007309C001F129F1271
:1002B0001B0880399B0083121F10941283160611AD
:1002C00086140612003083129400831694000108ED
:1002D000C73908388100831290010030F80092007D
:1002E00000308316920007309C0005080630F700A6
:1002F000F70B782900001C0883120D1383169D014B
:100300008F010F0883128B16C0308B041330A900A5
:0403100086296300D7
:04400E00193FFC3F1B
:00000001FF
